:020000040000FA
:1000000004309F009E009C01003065008501FF3098
:1000100066007F30620006080F399D000330061F1E
:100020009D061D080339031903309D040C30861FFB
:100030009D061D080C3903190C309D041E0804028E
:10004000FE39031D1D14031D9D141D1805101D1CD4
:1000500005149D1885109D1C85140430061E05305E
:100060001D1D09309D1D00309F001F081E02031C2E
:100070009E0A1E081F02031C9E03103085069C0961
:100080009C1C05159C18851510309A007A309B0031
:100090009B0B48289A0B46284D28051185118A305C
:1000A0009B009B0B512800001E08000000008207E7
:1000B000622863286C28762880288E289F28A82804
:1000C000B228BD280B281B309A000B309B009B0BDD
:1000D00067289A0B65280B2836309A000B309B0056
:1000E0009B0B70289A0B6E2800000B2851309A0049
:1000F0000B309B009B0B7A289A0B78287F280B28C3
:1001000056309B0006309A009B0B84289A0B84285B
:1001100089288A288B288C288D280B289C309B00C6
:1001200006309A0001309900013098009B0B962808
:100130009A0B9628990B9628980B96280B28133023
:100140009A008B309B009B0BA3289A0BA1280B28AD
:1001500026309A008B309B009B0BAC289A0BAA2868
:1001600000000B284C309A008B309B009B0BB6286C
:100170009A0BB428BB2800000B280511851106191D
:040180000B28BF2861
:02400E00F13F80
:1042000041006C0063006F0072002D0046005300F7
:104210003300200043006F007000790072006900D5
:104220006700680074002000320030003000360063
:1042300020004D002E00200043006F007600690032
:0A4240006E00670074006F006E004E
:00000001FF
